S105FFFEC0003D
S113C0008E00FFCE10008680A73918CE00001809D4
S113C01026FCCE10008600A7301F3080FC86C4E6C4
S113C02031E7043DCE271002DF00CE03E802DF0231
S113C030CE006402DF04CE000A02DD06CE1000C684
S113C04000BDD000C6FFCEC073BDD000D601CB303A
S113C050BDD000D603CB30BDD000D605CB30BDD08B
S113C06000D607CB30BDD000C6FFCEC07FBDD00008
S113C0707EC00A5370616E6E696E67203D20046D48
S105C080560460
S113D000183C36C1FF2747C1002715C105272AC18F
S113D010042204C101242FBDD05E20003218383907
S113D020C63FBDD0FCBDD0FCC60FBDD0FCC606BDFE
S113D030D0FCC601BDD0FC20E3BDD10ABDD0B818D8
S113D0403018A70020D6BDD0DABDD0AF20CEE60080
S113D050C1042604C6FF20C4BDD0630820F0C10467
S113D060260139C10D2604BDD07539BDD103BDD10A
S113D0700ABDD07C39BDD10ABDD08D398114272396
S113D080814027278154271F8100271139811323C9
S113D09012812723168153230E8167230086018082
S113D0A080200C86402008861420048654200037F3
S113D0B016CB80BDD0FC333981132204C60120185D
S113D0C081272206C6038014200E81532206C6023D
S113D0D080402004C60480544C3981002707811401
S113D0E0230286014AC1012712C10226048B402073
S113D0F00AC10326048B1420028B5439F72000BD87
S113D100D11839F73000BDD1183918CE0002B62035
S113D110002BFB180926F73918CE0800180926FC3D
S104D12039D1
S9030000FC
